:100000006329B200F839A400A40CA40C240C8407C2
:100010007320B20000055F293208031C03010006AB
:10002000320580065F29A01123080319A0150530A9
:10003000A2002730A900103029200330A900E830A1
:100040002920A90164302920A9010A3029202C087F
:100050003028A8002D08A5002C08A400FA202408A8
:10006000A400A2030319A011230803193A282202AD
:10007000031841282408031DA011A0194128303E6F
:10008000472808000C1E4228990003145F292119F3
:100090004228080083169B0083161C141A089B0A2A
:1000A0005F29A901A800FF30A807031CA907031CAA
:1000B0005F290330A500E5305F205328A501F63EF7
:1000C000A400A509031C6A28FE300000A407031839
:1000D0006528A4070000A50F6428000024187028D4
:1000E00024187228080000308A0032080739820775
:1000F0000134023404340834103420344034803461
:1001000027082F068039B100A71F9128A409A50947
:10011000A609A709A40A0319A50A0319A60A03191F
:10012000A70AAF1F9E28AC09AD09AE09AF09AC0AFA
:100130000319AD0A0319AE0A0319AF0AA801A901F0
:10014000AA01AB01B601B701B801B9012F082E040D
:100150002D042C040319DC282030B0000310A40D5A
:10016000A50DA60DA70DB60DB70DB80DB90D2F082D
:100170003902031DC5282E083802031DC5282D0885
:100180003702031DC5282C083602031CD6282C086C
:10019000B6022D08031C2D0FB7022E08031C2E0FCC
:1001A000B8022F08031C2F0FB9020314A80DA90DC4
:1001B000AA0DAB0DB00BAE28B11FE928A809A909FB
:1001C000AA09AB09A80A0319A90A0319AA0A03195B
:1001D000AB0A3608AC003708AD003808AE00390865
:1001E000AF002808A4002908A5002A08A6002B08AB
:1001F000A7005F29AD01AC011030B000250DAC0D9A
:10020000AD0D2808AC022908031C290FAD02031804
:1002100010292808AC0729080318290FAD07031077
:10022000A40DA50DB00BFE2824085F292030B000D6
:10023000B601B701B801B9010310241C2D292C08FF
:10024000B6072D0803182D0FB7072E0803182E0F19
:10025000B8072F0803182F0FB907B90CB80CB70C43
:10026000B60CA70CA60CA50CA40CB00B1C290800FE
:100270001030B300A501A401B10CB00C031C462939
:100280002808A40729080318290FA507A50CA40C02
:10029000AD0CAC0CB30B3C292C085F29A400A71BA8
:1002A000532124085F29A409A509A609A709A40ABE
:1002B0000319A50A0319A60A0319A70A080083133C
:1002C00083120313080083160F3099002030980022
:1002D000831280309800A001C23083168600FD3062
:1002E0008500073083129F009F2A861564305E20A8
:1002F000061464305E20861164305E20061064307F
:100300005E2008008615851464305E208611CC219D
:10031000DE21061BBF298519AD294D304220413011
:100320004220473042204E30422045304220543057
:1003300042203D304220203042200430A100A30161
:100340003A08AC003B08AD00132020304220422088
:10035000422042200D304220BE294D303A07C200D3
:100360003B080318013EC3004D3042203A084220AA
:100370003B08422042084220430842208929822922
:1003800085100830A400A40BC32908008514083088
:10039000A400A40BC92908000930C100C021C6214E
:1003A0003A3084004108003E012003100518031470
:1003B0000C200130C1020318CE290800C021C6213B
:1003C00083100518831483184014831C4010C02127
:1003D000C6218310051883148318C014831CC01011
:1003E000C021C62183100518831483184015831C6F
:1003F0004011C021C6218310051883148318C0152D
:10040000831CC011C021C6218310051883148318D2
:100410004016831C4012C021C62183100518831486
:100420008318C016831CC012861514305E20080085
:100430003A08B0003B08B1002D30A800A9013821CE
:10044000C6002D08C7004608C4004708C50007308D
:10045000A4000310C50CC40CA40B292A7F30460548
:10046000C800C9014808B0004908B1000A30A80016
:10047000A9013821C8002D08C9004808CA00490848
:10048000CB000730A4000310CB0CCA0CA40B432AEA
:100490007F304805C600C701C708031D532A4030F6
:1004A0004602031C612A4A08093A4B04031D5E2ACE
:1004B000C40A0319C50ACA01CB01612ACA0A031971
:1004C000CB0A080055085404031D672A08003A089F
:1004D000A4003B08A500A601A701AF01AE010430AE
:1004E000AD00AC0116212708D9002608D800250840
:1004F000D7002408D6005908A7005808A6005708B6
:10050000A5005608A4005408AC005508AD00AE0183
:10051000AF0180202708D9002608D8002508D70079
:100520002408D6005608BA005708BB0004303B0226
:10053000031C9E2AFF30BA000330BB0008000610DF
:100540000330A900E8305220CE01CC01CD010130AA
:100550004A20D4004C20D50003304A20DA004C2039
:10056000DB0086158514BA01BB0114305E20051925
:10057000BB2A75218229861114305E20CC2162228B
:100580008618E72A3B08AD003A08AC00AE01AF017F
:10059000013EBC00FC30BD002D0803182D0FBD0727
:1005A000FF30BE002E0803182E0FBE07FF30BF001D
:1005B0002F0803182F0FBF073F08A7003E08A6000B
:1005C0003D08A5003C084E21BA002508BB000230BA
:1005D0004E02031CF72A4C08A4004D08A5004E0843
:1005E000A800A901FA20D0002508D100FB2A4C0858
:1005F000D0004D08D1003B085102031C0E2B031DF7
:10060000052B3A085002031C0E2B3A085002D20068
:100610003B08031C013E5102D300162B50083A023E
:10062000D2005108031C013E3B02D300D308031D36
:100630001D2B04305202031C242B3A08CC003B082B
:10064000CD000130CE002F2B0F304E0203182F2B80
:100650003A08CC073B080318013ECD07CE0ADE213D
:1006600001305120C01D362B0612382B06160616F7
:10067000401E3C2B86123E2B86168616061B8C2BA4
:1006800085196C2B1822413042205A3042204930C3
:1006900042204D30422055304220543042204830D4
:1006A0004220203042203D30422020304220043081
:1006B000A100A3014408AC004508AD0013202E3072
:1006C0004220A3014A08AC004B08AD0013202030A3
:1006D00042200D304220892B41304C07B4004D0898
:1006E0000318013EB5004E083407C2003508031850
:1006F000013EC300413042204C0842204D084220B8
:100700004E0842204208422043084220CE01CC013C
:10071000CD01061B8C2B892BB12A63008D2B8F2BCF
:02400E00223F4F
:0A42000000000000000000000400B0
:00000001FF
